:020000040000FA
:020800001100E5
:10081000E8CFDCFFD8CFDCFFABA202D0AB98AB882F
:0E082000ABB4AE50F2A498EF20F0E7EF1EF05C
:10084000B4EC1EF059EC19F0140E84DDD8EC01F074
:10085000830EB2EC01F07D0EF76E340ED2EC18F080
:10086000C10EB2EC01F03E0ED2EC18F0CE0EB2EC9E
:1008700001F0300E6EBA310E6EBC320EB6EC01F0E5
:1008800069EC19F0E1EC1AF060EC19F0E9EC1CF0FD
:10089000400EB2EC01F0770EF76EB80ED2EC18F005
:1008A000800EB2EC01F0A4EC01F0DF6B01EC09F07A
:1008B00042EC1DF03BBEB5EF0AF033B4E8EF0AF0AE
:1008C0002DB0FED702AD09D001EC09F00CEC1AF006
:1008D00041EC07F071EC1BF0C1D020EE80F065EC2C
:1008E00006F09CD96FEC16F099D96BAECBD98DEC94
:1008F00018F0EFACEFBE3FDA3DAE02D09DD9EDD798
:1009000051EC08F014EC18F0CFB3F5EF04F0A4ECC0
:1009100017F089EC18F0EFAC13D081EC36F030B260
:1009200002D0DF6B17D09BEC17F001EC18F0C6EC8F
:1009300014F00FEC18F01CEC18F00EEC02F00AD0DA
:10094000318680EC36F0C6EC14F024EC18F02AB0B6
:100950009EEC1AF09EEC15F06EDB2EA020D02E90AF
:100960009EEC1AF001EE2AF002B101EE46F011EE13
:100970002AF002A111EE46F031DA880EB2EC01F055
:100980003E0EB6EC01F0410E02A1420EB6EC01F0B3
:10099000060E9FEC01F01AEC38F09EEC1AF0DCEC3D
:1009A00017F02DA211D001EE2AF002B101EE46F0AF
:1009B00011EE62F013DA028D01EC09F02EB40CECAA
:1009C0001AF09EEC1AF04AD0D7EC17F02DB26AEF6D
:1009D00013F06BAE82D73EBE29EF09F030B23BAECA
:1009E0007CD79EEC1AF0A0EF0FF0DF51D8B407D0FF
:1009F000DFAF41EC38F0DFBF48EC38F0DF6BCFB150
:100A00002FA016D055EC15F02B9026A507D0810EFF
:100A10001DEC15F02BB05CEC18F006D0010E1DECAF
:100A200015F02BB057EC18F024EC18F02F9011D0E3
:100A3000CE0EB2EC01F0FFDACFA70BD001EED1F071
:100A4000CFA301EED3F0ED3C04D0CF912F80C3ECC7
:100A500020F09EEC15F081EC36F03FD720EE80F0D0
:100A600065EC06F0DBD86FEC16F0D8D86BAE0AD97F
:100A70009B51615CD8B406D001EC09F00CEC1AF083
:100A800041EC07F08DEC18F0EFACEFBE74D93DAE41
:100A900002D0D2D8E3D751EC08F014EC18F0CFB55F
:100AA000BEEF05F0A4EC17F038EC15F024EC18F0CC
:100AB0002AB09EEC1AF02EB424D06DEC09F024D0AC
:100AC00089EC18F0EFAC13D081EC36F030B202D0E4
:100AD000DF6B17D09BEC17F001EC18F0C6EC14F0AC
:100AE0000FEC18F01CEC18F00EEC02F00AD0318676
:100AF00080EC36F0C6EC14F024EC18F02AB09EEC32
:100B00001AF09EEC15F097DADCEC17F02DA206D067
:100B1000029D41EC07F09EEC1AF0DFD63EAE0BD002
:100B2000029D9EEC1AF041D99EEC1AF051EC08F0AF
:100B30003EBEFED7D2D681EC36F030B208D027AF19
:100B400006D041EC07F02F9CDF6B2EEF05F0DF5154
:100B500005E001EC09F02EB40CEC1AF041EC07F0C2
:100B6000D7EC17F02DB26AEF13F06BAE77D730B237
:100B70003BAE74D79EEC1AF0A0EF0FF0DF51D8B463
:100B800007D0DFAF41EC38F0DFBF48EC38F0DF6B67
:100B9000CFBD1AD0CFB12FA004D0E7EC05F02F9035
:100BA00011D0CE0EB2EC01F046DACFA70BD001EE99
:100BB000D1F0CFA301EED3F0ED3C04D0CF912F8044
:100BC000C3EC20F09EEC15F081EC36F047D75EECDC
:100BD00002F05BEC02F0C70E226E64EC02F09B5157
:100BE000136ECF9B26A507D0C7DBCFAB09D0C80EAD
:100BF000136EC2DB05D0B8DBCFAB02D01368B4DB19
:100C000013509B6F0FDB0CEC1AF0A4EC17F014ECF4
:100C100018F042EC15F024EC18F012002C9802BDEC
:100C200007D002B12C8827BF30B212002C781200F6
:100C300063BD63AF1200F8D793EC17F08BEC18F09C
:100C400015EC18F0B0EC01F0780EF76E030ED2EC54
:100C500018F0140ED2EC18F0250ED2EC18F080EC3F
:100C600036F02D88C6EC14F02D98FEEC15F006EC4D
:100C700016F09FEC18F025EC18F014EC18F0A9EC25
:100C800015F01200DFEC39F0CFA5CFB310D051AC86
:100C900002D0269503D051AE1200268502ADD6ECC7
:100CA00037F002BD8FEC38F06B6A3090120051AA19
:100CB00005D0EFEC1BF02A80DF6BF6D751BC41EC7E
:100CC00038F051BE48EC38F0120029D851B2120069
:100CD000CFA3CFB5120002BD0AD0E1EC17F02DA2D0
:100CE00006D0027143D841EC07F09EEC1AF02EB208
:100CF0004BD8E6EC17F02DA209D08DEC18F0400E81
:100D0000EF26EF24D8B0EF6E2EEC38F0EBEC17F0B6
:100D10002DA2120089EC18F0EFAC21D02CD030823B
:100D200051B43092040E425CD8B0309230B210D040
:100D30002DBE09D07FEC18F00A0EEF6201D003D06F
:100D40000E0EEF6203D03082519402D030A2CF91C8
:100D500065DF1200519089EC18F0EFBC1200518051
:100D6000CF9389EC18F0EF8C2D8A1200519089EC0A
:100D700018F0EFAC1200518089EC18F0EF9C2D9A1E
:100D80001200519027BF120002BD09D0455102A1A7
:100D900061510A0804E0277F51809EEC1AF02E92E0
:100DA0001200519027AF1200EFD711D863BD63AF87
:100DB000120011EE2AF002A111EE46F001EE7EF0D3
:100DC0000DD83F0E2B174717278F28DF120011EE83
:100DD0002AF002B111EE46F001EE62F01C0E0FD8BF
:100DE00061394511066F526E120002EE22F012EECA
:100DF00008F004D002EE08F012EE22F01A0EEECF48
:100E0000E6FFE82EFCD71200276A03EE00F0B50ECD
:100E1000236E080E266ED8B120D8AD0E236E26069E
:100E2000D751376E37BE19D8F80E23263746260617
:100E3000F9E71200050E266E276A03EE00F0430E56
:100E4000236ED851376E37BA08D8F80E23263746A6
:100E5000262EF9D7D8BD01D81200EE6A040E256EF1
:100E60002350A3EC03F02650EE6EFC0E2326EE6A10
:100E7000040E256E2350A3EC03F0040E2326272A2C
:100E8000120014EC18F01AEC07F0266A274C21D057
:100E9000F1EC01F003EE05F02650E926EE502BECC4
:100EA00018F028EC18F00EEC02F066EC18F0D89070
:100EB0001432153216321732183201EC02F05BECA4
:100EC00003F0D8A4D8A001D004D00B0E2626272EDC
:100ED000DDD703EE05F02628E9262BEC18F05BECB5
:100EE00003F001E20CD003EE05F02650FB0FE926DB
:100EF0002BEC18F05BEC03F0D8A4D8A002D052EC95
:100F000018F003EE05F02650E926EE5084EC18F0B8
:100F1000EF6E84EC18F0EF502CE104EC07F0266A39
:100F200003EE05F02650E926EE502BEC18F05BECB2
:100F300003F005E20B0E2626272EF2D70CD003EE87
:100F400005F02650FB0FE9262BEC18F05BEC03F0C4
:100F5000D8A4D8A005D07FEC18F00E0EEF6E10D0FC
:100F600003EE05F02650E926EE507FEC18F0EF6E08
:100F700007D084EC18F0EF50080F7FEC18F0EF6EFC
:100F8000120052502CB8523802BD7D510F0B5C6ECE
:100F90002D9EF70F1AE3FB0F18E05C38276ED890F0
:100FA0002730710F276E1BEC19F014EC18F05BEC76
:100FB00003F001E209D02750040F1BEC19F05BECA1
:100FC00003F0D8A4D8A001D02D8E6FEC1EF02F9284
:100FD0000A0E5C6212002F8201EE2AF02CB801EE9C
:100FE00046F002BD01EE62F0050EEF6E120080ECDD
:100FF00039F0246E1BEC19F05BEC03F0D8A009D09B
:101000002450040F1BEC19F05BEC03F0D8A4D8A01B
:10101000120093EC39F0246E25EC19F02450040FE3
:101020001BEC19F00EEC02F0D8900F321032113296
:101030001232133212002CEC08F030B204D0020E3F
:101040009FEC01F01200020ECE03770EF76E980EA1
:10105000F324D2EC18F01200F1EC01F064EC02F091
:10106000C2B2FED70F0ECE6FFD0EA96EA69EA69C35
:10107000A680A850DC6EA92AA680A850C35CDD50CB
:10108000C45804E2FD0EA926CE2FF2D7A968CE29B6
:10109000D45DD8A0CF87D8B0CF97C28201EC02F040
:1010A0001200B0EC01F0520E30A2540EB6EC01F07A
:1010B000580EB6EC01F0B4EC01F002AD0DD05D506D
:1010C0004D0F5D66130FB6EC01F02D0E64BF070ED9
:1010D000B6EC01F08CD80FD0790EF76E840ED2ECFE
:1010E00018F0410E02B1420EB6EC01F0200E27BFFF
:1010F000730EB6EC01F0472C50D0000E90EC18F0B7
:10110000070EEF142FB2080E040D770EF76E000EC7
:10111000F3242F86D2EC18F02F96780EF76E8DEC14
:1011200018F0CFA3CFB50DD0EFBCEFAE02D0060EB6
:1011300031D0EFBE29D0EFBC29D089EC18F0EFBC3C
:1011400016D0B4EC01F0CFA908D04F0E26B5520E40
:10115000CFA1580ECFBD5B0E05D0490E26B54C0E63
:10116000CFA1550ECFB516D0CFA33D0E13D0080E8C
:10117000E926ED50EF10010EEFBE000ED8B4200EA0
:10118000B6EC01F0000E06D0010E01D0000EB6EC58
:1011900001F0030ED2EC18F01200B4EC01F00D0EC9
:1011A0005C6406D07A0EF76ECF0E5CB0D60E1CD003
:1011B000010E28A1030E9FEC01F000D052502CB874
:1011C00052380F0BD8902DB83430040D28B1030DD0
:1011D000770EF76E540E28B1240EF324D2EC18F0DB
:1011E000790EF76E000E28B1D2EC18F012005E50A6
:1011F000B6EC01F05F50B6EC01F06050B6EC01F0D7
:1012000012005EEC02F05BEC02F0C90E226E64ECA0
:1012100002F09B51136E2D8802ADC3EC14F002BD99
:1012200098D82D9813509B6F132AC80E136408D0BA
:10123000500E5E6E4C0E13A0550E5F6E200E07D042
:1012400099EC02F00C505E6E0D505F6E0E50606EA9
:101250001200A4EC01F02D862C902CB021D001ECD2
:1012600009F0B0EC01F0790EF76E4A0ED2EC18F0EE
:10127000BEDF0CEC1AF08DD82EA40ED001EE6CF06F
:1012800015EC18F000DEA4EC17F042EC15F0FEECC3
:1012900015F01FEC08F001D020D8DCEC17F02DB2CF
:1012A000A1EF0DF03EAE2D962DA63EAED6D74AEC60
:1012B0001AF06FD83850EF12A4EC1AF0AFEC0DF022
:1012C0009BC1DCFFE1EC1AF0DDCF9BF1A4EC01F057
:1012D000DF6B41EC07F0D3EF04F0C00EB2EC01F08D
:1012E000790EF76E3A0ED2EC18F012007EDD2C82E9
:1012F0000AD8120071EC1BF002EE21F0EF6A2C927A
:1013000002D878DD12005EEC02F05BEC02F0C70E52
:10131000226E64EC02F013689A6BCF9B25D8CFBB8A
:1013200013D02CB206D0020EFFEC19F0E8AE07D0B5
:1013300008D0040EFFEC19F00F0BD56302D09A2BE6
:10134000EDD73850EF1AEAD7CF9D010E9A65CF8DB1
:10135000120042EC15F013509B6F02D8DF6B1200A5
:10136000DF510FE0DFBF08D0132A222813600BD013
:101370000ED82EA4F9D705D0130605E308D82EA45D
:10138000FBD705D812009B51136ECF8BFAD71350A1
:1013900001D09B51376E070B236E374237423742DD
:1013A0001F0E3716800E386E232A3846232EFDD79F
:1013B00002EE08F03750E9262E943850EF14D8A4E6
:1013C0002E8412002C90DCEC17F02DA22CB028D02B
:1013D0005EEC02F05BEC02F00F0E226E64EC02F0A9
:1013E000D551136E2D88C3EC14F02D981350D56F82
:1013F0007DDFB0EC01F0790EF76EAC0ED2EC18F098
:10140000D5514D0FD567130FB6EC01F017D83EAE8E
:10141000DAD7CF95C9EC1AF0CF85E7EC05F09FDB62
:1014200080EC1BF0D5515D6E2D0E5E6E5F6E606EB2
:101430005DDF37DE03D814EC38F01200C00EB2ECDA
:1014400001F0CFAD06D0790EF76EBB0ED2EC18F0DE
:101450001200100E9FEC01F0120065EC0DF00F0E63
:10146000226E66510F0B136E18D8DCEC17F02DA20C
:101470002CB05ED01350376EC3EC14F013503762AB
:101480000CD83EAEF2D7F00E6617135066138DECF3
:101490001AF0D6EC11F063DB4BD0D6EC11F0135000
:1014A0004D0F1366130FB6EC01F0830FB2EC01F091
:1014B0000D0EB2EC01F012002D88C00EB2EC01F05E
:1014C0001FEC08F0220EB6EC01F04DEC16F0220EE7
:1014D000B6EC01F01FEC08F0356A42D864EC02F07B
:1014E0005EEC02F0200E1D6E5BEC02F07F0E226EB1
:1014F0002C90DCEC17F02DA22CB01AD001EE74F079
:101500003550EB50136E376EC3EC14F001EE74F0EF
:10151000355013C0EBFF135037621DD84BB40ED0BB
:101520003EAEE7D7628F8DEC1AF0D6EC11F017DBE8
:10153000D6EC11F02D980CEC1AF012001D6A070E73
:10154000226E35C013F0C3EC14F013C035F008D888
:101550004BB4F7D7C5D7D6EC11F01350B6EC01F069
:101560003550C30FB9EC11F0120063EC0DF0060E0C
:10157000226E2CB0A1EF0DF0C3EC14F0B0EC01F032
:101580007A0EF76E000ED2EC18F0D8EC0FF0C00E09
:10159000B2EC01F07A0EF76E1338090FD2EC18F0A6
:1015A000D7EC17F02DA2E5D7A4EC01F01328E84EF4
:1015B000A1EF0DF0E84E0CD0E84EE0D2E84E38D363
:1015C000E84EF4EF0EF0E84E5EEF0FF07AEF0FF01A
:1015D00063EC0DF02C96780EF76E1D0ED2EC18F021
:1015E0007A0ED2EC18F033C034F0030E136E020EF4
:1015F000226E3350E00BE8BE03D0E844132EFBD735
:1016000013C036F02CB099D233B0C3EC14F0C00E36
:10161000B2EC01F0090E1302790EF76E160EF324E8
:10162000D2EC18F01350D8B4EDD7D7EC17F02DA2A8
:10163000E9D7365033A413622C86100E126E124670
:10164000132EFDD76E501F0B12106E6EDF6B020E45
:10165000226E64EC02F06F30030B136E366E2CB604
:10166000136A2CB06AD2B0EC01F0780EF76E1D0E42
:10167000D2EC18F0830ED2EC18F0C3EC14F0C00ECC
:10168000B2EC01F0136609D0790EF76E160ED2ECAB
:1016900018F0050E9FEC01F00AD0780EF76E980E48
:1016A000D2EC18F0320E13A0340EB6EC01F0D7ECE9
:1016B00017F02DA2D6D7365013622C866F9213B036
:1016C0006F826F9413B26F84010E6FB2020E6FB40B
:1016D000040E356E010E226E64EC02F06EBA20D05C
:1016E0006FB61380A4EC01F0780EF76EA20ED2EC68
:1016F00018F00BDA13A014D0A4EC01F0780EF76EFA
:10170000B20ED2EC18F0C00EB2EC01F0780EF76E0B
:10171000C20ED2EC18F01AEC38F01AEC38F0E2D91C
:101720006F9613B06F86A4EC01F0050E6EBC060E2A
:1017300002EC03F043EC18F0060E02EC03F0120E7C
:101740006FB605D06EBC280E6EBE320E04D06EBCD5
:10175000320E6EBE3C0EF9EC02F048EC18F02CA6EE
:101760000DD0050E02EC03F01E0E6EBC640E6EBEB4
:10177000640EF9EC02F052EC18F003D0040E25ECE4
:1017800019F0F1EC01F02CB0D8D1B0EC01F0780EEA
:10179000F76E1D0ED2EC18F0210ED2EC18F080EC92
:1017A00036F0C6EC14F0FEEC15F0D7EC17F02DA2D5
:1017B000EAD7FEEC01F05BEC03F0D8A42C86F1EC48
:1017C00001F0F1EC01F0F1EC01F05CEC18F0880EA6
:1017D000B2EC01F0780EF76ED20ED2EC18F0FEECFF
:1017E00001F033EC03F061EC02F0060E6EAA140E69
:1017F000186E66EC03F0050E6EAA030E186E43EC2D
:1018000018F06EEC03F070EC18F02CA606D0010E68
:101810006EBC040E6EBE050E02D06E501F0B136E12
:10182000366E2CB08AD142EC15F0C3EC14F02C8249
:10183000C00EB2EC01F02C941D50136204D0010EC6
:10184000136E2C9233D0FEEC01F0EEEC01F0F1ECD3
:1018500001F01350F9EC02F052EC18F0060E02EC15
:1018600003F0030E6EBC080E6EBE0A0EF9EC02F019
:101870005BEC03F0D8A02C842CA46EAE15D0050E22
:1018800002EC03F0FF0EF9EC02F05BEC03F0D8B0D1
:101890000BD0060E02EC03F0100EF9EC02F05BEC3C
:1018A00003F0D8B0D8A42C8401EC02F098EC02F03C
:1018B0000D50B6EC01F00E50B6EC01F07D0EF76E57
:1018C000200ED2EC18F0CD0EB2EC01F0780EF76ECF
:1018D000460E2CA43D0ED2EC18F0D7EC17F02CA439
:1018E0002DA29FD7365013622C86E00E6E16135031
:1018F0006E122C8A646AFEEC01F01350F9EC02F0CF
:1019000052EC18F010EED8F02EEC18F00A0EF9ECAC
:1019100002F0EEEC01F06F90060E02EC03F0190EEF
:10192000F9EC02F05BEC03F0D8B06F802CA26F9062
:1019300033A0339242EC1DF061EC02F00A0E186EF7
:1019400033EC03F066EC18F001EC02F033B061EC1C
:1019500002F019EC02F06BEC18F00EEC02F00EEC59
:1019600002F070EC18F019EC02F02CB607D0080E5B
:101970000DEC19F052EC18F054EC0DF0B0EC01F055
:10198000780EF76E1D0ED2EC18F08E0ED2EC18F019
:1019900080EC36F0C6EC14F0F1EC01F0FEEC15F042
:1019A00054EC0DF0060E02EC03F057EC16F001ECCF
:1019B00002F0D7EC17F02DA2E1D72C9A66EC18F0C4
:1019C00054EC0DF0F1EC01F054EC02F075EC1CF06D
:1019D00000EEE2F066EC02F0A4EC01F000EED8F0CC
:1019E0002BEC18F0090EF9EC02F052EC18F061EC57
:1019F00002F0140E186E33EC03F070EC18F05EEC8D
:101A000002F02CA60BD0050E02EC03F0320E6EBCD9
:101A1000AF0E6EBED20EF9EC02F006D00D0E1BEC2E
:101A200019F03550F9EC02F052EC18F02C902CB073
:101A300084D0B0EC01F0780EF76E700ED2EC18F096
:101A40001C0ED2EC18F0250ED2EC18F080EC36F01B
:101A5000C6EC14F0FEEC15F0D7EC17F02DA2E7D78A
:101A600061EC02F03550186E33EC03F0F1EC01F04C
:101A70003BD813B007D020EE80F034C033F059ECDF
:101A800019F073D501EC02F00D0E24EC19F001EC05
:101A900002F0080E11EC19F001EC02F0040E24EC37
:101AA00019F058EC19F061D566EC18F064EC02F00E
:101AB00054EC02F00A0E6FB2140E6FB4280E076ECB
:101AC00034EC03F01200A4EC01F02D882C9064ECAF
:101AD00002F061EC02F05EEC02F05BEC02F012004E
:101AE0002E8A02D02E882E8663EC0DF0222A2EB884
:101AF0001380790EF76E660E2EB6750E2EBA570E3F
:101B0000D2EC18F02E962E982E9A2CB011D0C3EC51
:101B100014F0C60EB2EC01F0780EF76E460E13B05C
:101B2000430ED2EC18F0D7EC17F02DA2EED712002E
:101B300093EC20F02C90136A120034C033F059EC6F
:101B400019F0E1EC1AF0A4EC01F041EC07F02D984B
:101B50002F9CDF6B02AD6DEF04F02EEF05F003D884
:101B600045BEFED71200A4EC01F0850EB2EC01F0E8
:101B70007A0EF76EC90ED2EC18F01200346A64ECDB
:101B800002F005D061EC02F0182A0EEC02F06BECCA
:101B900018F034B008D0760EF76E2A0ECDEC18F09F
:101BA00048EC18F011D0130E346005D0000EF76E1B
:101BB000710E25EC19F0000EF76E0D0E1BEC19F0EE
:101BC0000EEC02F070EC18F0000EF76E3444E844AE
:101BD000710F25EC19F02CB0A1EF0DF0B0EC01F075
:101BE000DEEC08F0780EF76E670ED2EC18F06D0E92
:101BF00034B0700ED2EC18F006EC16F080EC36F033
:101C0000C6EC14F0FEEC15F02DA204D04150F90FF3
:101C1000D8B42871D7EC17F02DA2DDD73444E844AE
:101C2000710F24EC19F0342A1C0E3462ABD79DD40A
:101C3000346A356A2C962F8C64EC02F0F1EC01F0DA
:101C4000000EF76E710E0ED034B015D061EC02F0BC
:101C5000182A0EEC02F0F1EC01F0000EF76E34449D
:101C6000E844B10F25EC19F070EC18F001EC02F02B
:101C70006BEC18F022D0070E02EC03F0070EF9EC23
:101C800002F048EC18F00A0E34600ED0000EF76E29
:101C90003444E844B50F25EC19F061EC02F0182A41
:101CA00019EC02F070EC18F0000EF76E3444E844C2
:101CB000B10F25EC19F06BEC18F0000EF76E344400
:101CC000E844170F25EC19F02CB0A1EF0DF076D8F1
:101CD0006D0E34B0700ED2EC18F0040E9FEC01F0D3
:101CE00080EC36F0C6EC14F0FEEC15F0D7EC17F0F3
:101CF0002DA2EAD73444E844170F24EC19F034B08D
:101D000006D8342A0C0E34629FD72F9C2ED4F1ECC7
:101D100001F0070E02EC03F0070EF9EC02F048ECBC
:101D200018F045EC02F043EC18F03444FC0B470F7C
:101D300025EC19F02CB03ED041D8150ED2EC18F09D
:101D400081EC36F0C6EC14F0FEEC15F0D7EC17F091
:101D50002DA2F0D7000EF76E3444FC0B470F24EC95
:101D600019F02C86050E02EC03F0530EF9EC02F08C
:101D700048EC18F045EC02F043EC18F035505F0FDA
:101D80002FEC19F02CB016D019D8150ED2EC18F093
:101D900081EC36F0C6EC14F0FEEC15F0D7EC17F041
:101DA0002DA2F0D7000EF76E35505F0F2EEC19F014
:101DB000030E352601EC02F02C961200B0EC01F077
:101DC000D8903430D8B4080E040D770EF76E740E28
:101DD000F324D2EC18F0780EF76E1C0E2CB60A0E17
:101DE000D2EC18F0150E1200010E346E5BEC02F00E
:101DF0002268030E216E5EEC02F007D061EC02F067
:101E0000182A0EEC02F06BEC18F0000EF76E34445A
:101E1000DF0F50EC19F0B0EC01F0780EF76E6D0E9C
:101E2000D2EC18F0B4EC01F0770EF76E980E342473
:101E30003424D2EC18F0780EF76E2A0ED2EC18F09B
:101E4000C60EB2EC01F02EAE04D0040E9FEC01F0F1
:101E500019D02EAC13D064EC02F0186AC2B2FED7CF
:101E6000C3501026C4501322000E1222420E90ECD2
:101E700020F0C282182EF2D7106A2E9CC3EC14F008
:101E800045EC16F0F1EC01F08FEC06F014EC18F0D4
:101E9000A9EC15F0B7EC1DF001EC02F0D7EC17F04F
:101EA0002DA2B9D7000EF76E3444DF0F4FEC19F0B6
:101EB000342A100E3462A2D7B5EF0AF014DE13A054
:101EC000B5EF0AF0400E266E1F0E146E000E156E52
:101ED00000EE0BF0040E256E1550A96EA4EC03F075
:101EE00000EE0BF0040E256EC1EC1AF0262EF0D792
:101EF000B5EF0AF01F0E146E030E156EE3EC19F029
:101F0000D8B4B9EF0AF0EFDD13A0B5EF0AF0400E38
:101F1000266E1F0E126E000E136E1350A96E00EE89
:101F20000BF0040E9EEC1BF02A8200EE0BF0040E68
:101F3000256EA4EC03F0040E1326262EEED7FF0028
:101F400063EC0DF0090E226E2CB0A1EF0DF0C3EC86
:101F500014F0B0EC01F07B0EF76E000ED2EC18F02E
:101F6000D8EC0FF0C00EB2EC01F01BD8D7EC17F094
:101F70002DA2EAD7A4EC01F01328E84EA1EF0DF052
:101F8000E84E27D0E84E87D0E84EE9D0E84E3CD165
:101F9000E84E10D2E84EA6D2E84E28D3E84E4FD3F2
:101FA00088D37B0EF76E13380B0FD2EC18F01200AB
:101FB000132A99EC02F0300E0D6403D00D50B6ECEC
:101FC00001F00E50B6EC01F0200EB6EC01F0130655
:101FD000120063EC0DF0030E02EC03F0050EF9ECB9
:101FE00002F048EC18F045EC02F043EC18F0346ACB
:101FF000000E90EC18F0EFCFDCFFEF6AB0EC01F0D0
:10200000780EF76E0E0ED2EC18F0B0EC01F0344002
:10201000070B95D8B4EC01F08FEC06F0349030A2A9
:102020003480840EB2EC01F0520E34B0540EB6EC93
:1020300001F03450050DF35003EEB0F0E92628EC22
:1020400018F081EC36F0C6EC14F0FEEC15F03450CC
:10205000050DF35013EEB0F0E1262EEC18F014EC61
:1020600018F0A9EC15F02F8EB7EC1DF02F9ED7ECD1
:1020700017F02DA2D1D7020E3426000E90EC18F0E6
:10208000EF2A34A8C2D7D9EC1AF0000E90EC18F061
:10209000DDCFEFFF55D7D6C135F063EC0DF02280D0
:1020A000346AC00EB2EC01F07B0EF76ECB0ED2ECB0
:1020B00018F0C30EB2EC01F0345041D82CB0A1EFAF
:1020C0000DF0136A35B01380C3EC14F0050E3462C2
:1020D00002D0D8B51380359013B03580B0EC01F044
:1020E0007B0EF76EAB0E13A0BB0ED2EC18F0D7EC44
:1020F00017F02DA2E3D73542342A34A6DAD735506B
:10210000D8A402D006D8C9D735C0D6F1C9EC1AF088
:1021100017D7A4EC01F045BAFED7B0EC01F07A0E67
:10212000F76EA90ED2EC18F0C00EB2EC01F07A0EE8
:10213000F76EB90ED2EC18F01AEC38F012002C92AF
:102140002FB42C82040D770EF76E010EF3242F941A
:102150002F86D2EC18F02F962CB22F841200D7C104
:1021600035F0D8C136F063EC0DF02280346AC00E31
:10217000B2EC01F07B0EF76EDB0ED2EC18F0C70E5E
:10218000B2EC01F03450040D770EF76E540EF324C8
:10219000D2EC18F02CB0A1EF0DF0136A35B013801B
:1021A000C3EC14F0359013B03580B0EC01F07B0E29
:1021B000F76EAB0E13A0BB0ED2EC18F0D7EC17F0F5
:1021C0002DA2E8D71DD8342A0D0E3464D8D718D8DC
:1021D00017D836503F0B3510D8A402D09ADFC3D79A
:1021E000369C3650010B3510D8A4368C36B4D68BBD
:1021F000368C35C0D7F136C0D8F1C9EC1AF0A0D66C
:10220000353036323532120063EC0DF02C942C96BA
:10221000B0EC01F07B0EF76E4B0ED2EC18F0C00E56
:10222000B2EC01F0780EF76ED60ED2EC18F0000E7C
:1022300082D820EE80F02CB408D05F0E226E34508D
:102240004CEC11F0346277D811D0226835504CEC48
:1022500011F035627BD8D7EC17F02DA207D012EE23
:1022600040F03506345035C0E3FF04D0E1EC17F000
:102270002DA202D02C9478D8EBEC17F02DA202D02E
:102280002C8472D82EACD5D791D82EDC13A058D67A
:1022900066DCD1EC1AF054D6386E64EC02F038509B
:1022A000136E2CB606D0C3EC14F0CAEC17F02DA2B6
:1022B0003CD02C90F1EC01F064EC02F098EC02F0D0
:1022C00060D8020E2CB4030E296E67D854D806D0FD
:1022D0002CB028D0CAEC17F02DA2FAD761EC02F08E
:1022E0000A0E186E12EC03F000EE0AF028EC18F05B
:1022F00041500F0B186E300FB6EC01F00EEC02F0EF
:10230000292EE6D7FEEC01F02CA62CB402D01366E1
:10231000130642EC15F0DF6B1350386E97EC11F09A
:102320003850120001EC02F0F4D7135012002CB612
:1023300011D02CB40BD0346E132A21D812EE40F0F9
:102340003450E328136E02D82C940ED0356E2C84B2
:1023500016D80AD02CB404D0356E2C9410D826D0C0
:10236000356E2C840CD822D0840E2CB48D0E2CA665
:10237000400FB2EC01F00E0EB2EC01F0120099EC3D
:1023800002F00BD80C502CB4B6EC01F00D50B6ECAA
:1023900001F00E50B6EC01F0120008D8840E2CB4F7
:1023A0008D0E2CA6400FB2EC01F012000C0EB2EC18
:1023B00001F0120063EC0DF02280C00EB2EC01F0CF
:1023C0007B0EF76E5B0ED2EC18F0136AD9A1138066
:1023D0002CB0A1EF0DF0C3EC14F0B0EC01F07A0ECC
:1023E000F76E790E13A0890ED2EC18F0D7EC17F027
:1023F0002DA2EED7D99113A0D98167D8DAAF04D036
:10240000060EDA6F200EDB6FD9B135D063EC0DF01C
:102410002C86B0EC01F07A0EF76E990ED2EC18F023
:10242000DA51136E99DFDB51136E9ADF060E02EC60
:1024300003F052EC18F020EE80F05EEC02F0070E94
:1024400002EC03F048EC18F0C6EC14F0FEEC15F0CA
:10245000F1EC01F0460EAAEC01F0E1EC17F02DB220
:102460000DD8EBEC17F02DB21DD801EC02F0D7EC33
:1024700017F02DA2E0D7C9EC1AF062D565EC0DF08B
:102480001D80100E226E2C946FDF2CB009D0CAEC88
:1024900017F02DA2FAD7DA514CEC11F0DA6F15D8FB
:1024A0005BDF120065EC0DF01D8022682C845CDF80
:1024B0002CB009D0CAEC17F02DA2FAD7DB514CECA6
:1024C00011F0DB6F02D84CDF1200E8CFDCFF010E09
:1024D000E66FEA6FE16FFA0EAAEC01F0DF6BDDCF79
:1024E000E8FF1000356AA4EC01F0790EF76E840E57
:1024F00035B2870ED2EC18F074D8EF5035B007D053
:10250000376E020E1D6E640E226E8A0E0CD0136E94
:102510003768372AFB0E1326D8B0FBD7010E1D6E85
:10252000330E226E950ED2EC18F02CB0A1EF0DF008
:1025300064EC02F03750136EC3EC14F01350376E96
:10254000C40EB2EC01F035A00ED0330E136207D0EA
:10255000790EF76EA40ED2EC18F0136817D0135052
:1025600013461346132699EC02F00C50B6EC01F01A
:102570000D50B6EC01F02E0EB6EC01F00E50B6EC9C
:1025800001F0790EF76EA00ED2EC18F0D7EC17F030
:102590002DA2CBD726D81350EF6EC9EC1AF0352AEE
:1025A00035A4A1D70F0E226E64EC02F0A4EC01F06A
:1025B0002CB0A1EF0DF0B0EC01F07A0EF76EDD0E4D
:1025C000D2EC18F0D451136EC3EC14F01350D46F46
:1025D00025EC38F0D7EC17F02DA2EAD7C9EC1AF0A9
:1025E000AFD401EED0F03550E9261200DADC020E4D
:1025F000226E2CB0A1EF0DF064EC02F011BD13803F
:1026000011BF1382C3EC14F0119D13B0118D119FF3
:1026100013B2118F13441326C00EB2EC01F0790EE1
:10262000F76E060E1324D2EC18F00F0ED2EC18F051
:10263000D7EC17F02DA2DDD7FBEC1BF081D4356A67
:10264000A4EC01F0780EF76E320E35B0300ED2ECFD
:1026500018F0350ED2EC18F0010E226E64EC02F088
:1026600035B003D00BBD138002D00BBF13802CB04C
:10267000A1EF0DF0C3EC14F0C00EB2EC01F0780E37
:10268000F76EE60E13B0EA0ED2EC18F0D7EC17F0A6
:102690002DA2EDD735B004D00B9D13B00B8D03D018
:1026A0000B9F13B00B8F352A35A2CAD7ABEC1AF0AB
:1026B00047D473EC0DF013A043D4146A156A0E6866
:1026C0000D680C680B6800EE0BF0040E256EC1EC73
:1026D0001AF0FF0063EC0DF00A0E226E62C013F0D8
:1026E0002CB0A5EF13F0C3EC14F01350626EB0ECF5
:1026F00001F07C0EF76E000ED2EC18F0D8EC0FF063
:10270000C00EB2EC01F038D91AD9D7EC17F02DA2CF
:10271000E7D7A4EC01F030D9010E226E1328136A1A
:10272000E84E13D0E84E15D0E84E24D0E84E2DD018
:10273000E84E3CD0E84E53D0E84E82D0E84EA2D0CE
:10274000E84EABD0E84EB4D0D3D0A8EC38F0A7EF29
:102750000DF0020E90EC18F0EFAA13802CB0F5D714
:10276000020E90EC18F0EF9A13A0EF8ADAD82DA29F
:10277000F5D7EBD704BB13802CB0E7D7049B13B07D
:10278000048BCFD82DA2F8D7E0D7020E90EC18F02A
:10279000EFB813802CB0D9D7020E90EC18F0EF9858
:1027A00013B0EF88BED82DA2F5D7CFD7228204A1CF
:1027B000138004A313822CB0C8D70481048313B000
:1027C000049113B20493D1D87C0EF76E1344E844FD
:1027D000D20FD2EC18F0ADD82DA2EDD7B6D70CD8C9
:1027E0002CB0B3D7C2D813B013D813A00CD804D8C8
:1027F00099D82DA2F5D7A9D713908DEC18F0EFA892
:10280000EFB6138012008DEC18F0EF98EF961200DF
:102810008DEC18F0EF88EF86760EF76EB80EF66E38
:10282000000E90EC18F0EF50070B0BBD080F0BBF1C
:10283000100FF6268DEC18F00800F550EF16120078
:10284000228226A1138026A313822CB07ED7268154
:10285000268313B0269113B2269387D87C0EF76E89
:10286000C20E13B013A204D0CA0ED2EC18F006D0D8
:10287000D2EC18F01350310FB6EC01F05AD82DA25B
:10288000E4D763D728B313802CB05FD7289313B055
:10289000288347D82DA2F8D758D705BF13802CB06E
:1028A00054D7059F13B0058F3CD82DA2F8D74DD72C
:1028B00084EC18F0EF509DEC1EF0346E2751341468
:1028C0003F0BD8A413802CB040D7345013B027133B
:1028D000341C13A0271749D87D0EF76E000E13A0E5
:1028E000100ED2EC18F0D7EC17F02DA2ECD72DD7A4
:1028F000228208BD138008BF13822CB026D7089D02
:10290000089F13B0088D13B2088F2FD87C0EF76E76
:102910001344E844BE0FD2EC18F00BD82DA2EDD72B
:1029200014D723D87C0EF76EBE0E13B0CE0ED2ECA9
:1029300018F00C0E9FEC01F0D7EC17F01200F1EC40
:1029400001F08FEC06F001EC18F089EC18F0EFBC08
:1029500030A264EC02F01CEC18F00EEC02F0F9D896
:10296000B7EC1DF001EC02F01200E9DFC3EC14F04B
:10297000C00EB2EC01F012007C0EF76E13380E0F91
:10298000D2EC18F0120091D82D8C53D08ED86BBE9B
:1029900049AE4FD0F1EC01F0B0EC01F0780EF76EDB
:1029A0005E0ED2EC18F0040E9FEC01F08AD8CE0E29
:1029B000B2EC01F01FEC08F0D7EC17F02DB22DBAF5
:1029C00003D069D82F7A7DD866D8DF5117E0DFBFF2
:1029D0000DD0EF06EFBEEF6AEF50F90FD8A40ED07E
:1029E00001EC02F0F1EC01F009D908D0180E2DBA73
:1029F000020E2CBA050EEF2AEF60EF6E4CD8DF6B9B
:102A0000080EEF6006D0EF50A6EC39F0B9EC11F0EB
:102A100005D062D847DBD6EC11F0F0D849BECCD750
:102A2000D6EC11F0A4EC01F001EC02F046D82EEC4B
:102A300038F0DF511CE0DF6BCF91266E2CD8E86AAE
:102A40002DBC04D0080EEF6004D0EF5002EC03F070
:102A500001D042D826AE03D045EC02F0266C0EEC35
:102A600002F02DBC04D0262EFAD72FBA47D825D88D
:102A70002D9C08D889EC18F0EFAC2DB8120025EC8D
:102A800037F0120039EC18F06EEC03F03EEC18F061
:102A900066EC03F01200030E90EC18F02DBA00EE75
:102AA00063F02DB800EE64F01200F5DF2F9A2DBA16
:102AB00002D0EFBE2F8AEF9E1200EDDF2FBAEF8E0D
:102AC00012008D0EB2EC01F0780EF76E3D0E2FBAAB
:102AD000400ED2EC18F01200EF6205D0760EF76EC1
:102AE000000E5BDB1200EF5CE806D890E834236E42
:102AF000760EF76E040E232434DB12000FAE03D0E3
:102B00003AEC02F02A8614BE45EC02F0EEEC01F03D
:102B1000D890143215321632173218320EEC02F0F9
:102B2000FEEC01F033EC03F012EC03F000EE0AF0DF
:102B30008FDA2AB63AEC02F02A961200F1EC01F094
:102B400008D8B7EC1DF001EC02F010EEDDF086DAEB
:102B500055D0000E90EC18F0070EEF140A0DF3504C
:102B600030A2050F03EEB0F0E9262BEC18F00EECC6
:102B700002F030B21CD0030E84EC18F0EF025F0EAE
:102B8000F3243CEC19F00EEC02F00E0E90EC18F071
:102B900054DAEF0EE926EFBEEFAC03D052EC18F09A
:102BA00006D0EFBE0EEC02F0EFBC19EC02F000EE26
:102BB000E2F051DA5BEC03F020E010EEE2F04EDAE6
:102BC000C1EC07F0040E84EC18F0EF02470EF3247A
:102BD0001BEC19F00EEC02F00FBE3AEC02F0000E06
:102BE000F76E0D0E1BEC19F066EC03F0080E0DEC01
:102BF00019F012EC03F075EC1CF01200C00EB2ECF0
:102C000001F002BD62AF06D001D847D8030E9FEC99
:102C100001F012002A960FAE03D02A863AEC02F099
:102C200099EC02F000EE07F02FAC2CBA00EE06F0A3
:102C3000080E2FBC090E256E2A98EF50B6EC01F055
:102C40002AB80CD0060E255C2E0ED8B4B6EC01F0D6
:102C5000030E255C2E0ED8B4B6EC01F0E92A252E21
:102C6000ECD72CAA03D0EF50B6EC01F02AB63AEC20
:102C700002F0790EF76E000E31B0030E2AA8D2ECE6
:102C800018F0B4EC01F02A96120099EC02F0040E50
:102C9000256E2A8800EE0BF0D0D701EE74F0080EF6
:102CA000256EEE50B8EC01F0252EFBD71200EEECAD
:102CB00001F000EEE2F0CFD95BEC03F003E1FEECB3
:102CC00001F01200FEEC01F010EEE2F0C7D910EEB8
:102CD000DDF0C4D912EC03F075EC1CF0120030A04A
:102CE00002D0519230906650655CD8B4120000EE6C
:102CF000C4F06550E926E926E926E926E926ABD99C
:102D00006550010F030B656E4F6A00EC3AF0185CDA
:102D100006E04F50030F4F6E5D08F7E112002EECF6
:102D200038F0F1EC01F04F2A00EF3AF0519051B237
:102D300091D05182060E256E00EEBEF050EC02F0EE
:102D4000070E256E00EE3BF050EC02F0518082D071
:102D50000A6A14500B6E0F08D8B4D8D015500C6EF8
:102D600016500D6E17500E6E6CEC02F089EC18F0D8
:102D7000EFBC04D025EC37F067D9C8D030A2C6D05C
:102D80005BD919EC02F0D7D87DDEAAD0C1EC06F0F1
:102D900061D000EEDDF05CD975EC02F00B50BFD8CD
:102DA0000C50BDD80D50BBD80E50B9D8010ECAD9A1
:102DB000B7EC39F0E7A8E7B6E88EB1D8A9D0AAEC0D
:102DC00006F048D0000E90EC18F0EFCFE7F0F80EC8
:102DD000EF16CAEC39F02FB2050EEF1214DD7EECBF
:102DE00037F0D8A0E7C0EFFF91D0519051B432D066
:102DF000518451802FD002BD89D08DEC18F0EF8C1A
:102E0000EF9E14BCEF9C14BCEF8E14BEEF9C7ED0E2
:102E10007DD07CD07BD0E1EC1AF0029DCF95CF9392
:102E2000CF9974D0519030A215D0518013D05190C9
:102E300051A210D0519251800DD0027167D0D1ECC7
:102E400006F008D0B6EC06F005D0519051A402D09F
:102E500051945180E86A51A0F00E61D859D0519434
:102E600055D0000E5CD85BD85AD859D858D857D806
:102E700056D855D854D84CD0000E51D849D0B2ECC1
:102E80001BF04DD8154A142AB2EC1BF048D840D09C
:102E90001650B6EC1BF0154A142A1750B6EC1BF06E
:102EA00035D030B205D0370E3AD8690E38D830D088
:102EB000000E35D82DD02AD0CE5130A2FF0E2FD8FB
:102EC00027D02A961450D8A42A8654EC02F0165023
:102ED0000D6E17500E6E6CEC02F02AB63AEC02F052
:102EE0009ED814D0000E27AFE88A30B2FF0E17D854
:102EF0000FD00A6A14500B6E15500C6E16500D6EE2
:102F000017500E6E6CEC02F01AD99FD8000E07D83D
:102F100001EC02F012002883F9D72893F7D79EA876
:102F2000FED7AD6E1200760EF76E260E36D9B0D8EB
:102F30005EEC02F01200760EF76E240E12D9A8D8BD
:102F400045EC02F0A0D81200F1EC01F084EC18F08E
:102F5000EF44E844E844170FDC6E77D9BCD8DD5065
:102F6000040F73D9BDD801EC02F01200EDDF0E0E94
:102F70005C601200F1EC01F05C44E844E844710F3D
:102F8000276E63D9A8D8040E27245FD9A9D801ECED
:102F900002F0120051B233D02DB405D0040E405CC3
:102FA000D8B02D842AD04050D8B42D9428D000EE2B
:102FB0003BF010EEBEF013D000EE3EF010EEC1F08C
:102FC0000ED000EE3FF010EEC2F009D000EE3DF062
:102FD00010EEC0F004D000EE3CF010EEBFF051B2A5
:102FE0000ED0E750236EEF5CEF50EFCFE7FF07E224
:102FF0002350040804E223502B082D82D8A02D92E0
:103000001200080E8DD810EE12F00F6A106A116AC5
:1030100071D812AE1200116810680F681200080E05
:1030200091D800EE12F066D07AD810EE10F00F6A48
:103030005DD810BE0F68120072D810EE15F0146A39
:1030400055D815BE146812007CD800EE10F04ED092
:1030500010EE0FF049D010EE14F046D000EE0FF055
:1030600043D000EE14F040D000EE05F010EE14F066
:103070003BD000EE19F010EE14F036D000EE1EF04A
:1030800010EE14F031D000EE14F010EE19F02CD048
:1030900000EE14F010EE1EF027D000EE05F010EE5A
:1030A0000FF022D000EE14F010EE0FF01DD000EE65
:1030B00019F010EE0FF018D000EE1EF010EE0FF029
:1030C00013D000EE0FF010EE05F00ED000EE0FF072
:1030D00010EE14F009D000EE0FF010EE19F004D04D
:1030E00000EE0FF010EE1EF0EECFE6FFEECFE6FFA3
:1030F000EECFE6FFEECFE6FFEECFE6FF1200DC6E8E
:103100001B0E0ED8DD501200DC6E1A0E09D8DD50F1
:103110001200020E05D00E0E03D0010E01D00A0ED1
:1031200002BD06D001EE2AF02CB801EE46F005D023
:1031300001EE62F02CB801EE7EF0E92612000E0ED0
:1031400001D00A0E02BD06D011EE2AF02CB811EE05
:1031500046F005D011EE62F02CB811EE7EF0E126BB
:103160001200F66E146A156A166A00EE17F04ED059
:1031700003EEAFF0EE6A760EF76E500EF66E100E9E
:10318000256E0900000EF5BEFF0EEE6EF5CFEEFFC8
:1031900003EC19F0252EF5D71200F66E146A00EE36
:1031A00015F02ED0F66E0900F550E89E2FA607D038
:1031B000236ED8A403D02FA4200E01D02350B6EC48
:1031C00001F0F5AEF0D71200740EF76EF00EF66E49
:1031D00000EE72F00CD0740EF76EF70EF66E00EE85
:1031E00072F00900F5CFEEFF0900F5CFEEFF090000
:1031F000F5CFEEFF0900F5CFEEFF0900F5CFEEFFAA
:103200000900F5CFEEFF0900F5CFEEFF0900F5CF7D
:10321000EEFF0900F5CFEEFF1200236E00EE14F072
:1032200004D02A82236E00EE0FF0050E256E235087
:10323000A3EF03F02A82236E146A00EE15F0040E49
:10324000F5DF15BE146812002A82236E0F6A00EEA5
:1032500010F0040EEBDF10BE0F6812002A82236EFE
:103260000F6A106A00EE11F0030EE0DF11AE1200DB
:103270000F68106812002A82236E146A156A00EE25
:1032800016F0030ED3DF16AE120014681568120094
:10329000236E146A156A166A00EE17F007D02A82A8
:1032A000236E0F6A106A116A00EE12F0020EBED78A
:1032B0002A8200EE6EF0040E256E000EA3EF03F0DE
:1032C00003EEAFF0EF3C1200B8EC18F0D9EC1AF0B6
:1032D000120061EC02F077D808E0080E256EE86A6B
:1032E000AAEC01F0252EFBD71200156A236A680E9E
:1032F000266E76D85B0E156E010E146E3FD8E10E69
:10330000156E020E146E3AD8800E156E000E146EF5
:10331000820E4DD87D0E156E000E146E840E47D8A9
:10332000F30E156E010E146E760EF76E4C0EF66EE1
:10333000010E29D8A5EC1EF034D9C00E116F800EF5
:10334000026F0E0E066F07D90A0ED06FD26F640E91
:10335000D16FD36F090ED46F770ED66FFF0ED76F74
:10336000C10ED86FFE0ED96F060EDA6F200EDB6F1E
:1033700010D9B8EC18F0D9EC1AF01200760EF76EEE
:10338000340EF66E060E256E040E376E3750246E20
:103390000900F55034DA154A142A242EF9D737508B
:1033A0001A081526000E1422252EF0D71200376EAB
:1033B0001E0E256E375023DA1A0E1526000E142223
:1033C000252EF8D7120032DA186E152A2FDA1816C1
:1033D000152A2CDA1816152A29DA1814010F1200EA
:1033E000400E256E2BDA235031DA154A142A252E89
:1033F000FAD75CDAA8EC01F0262EF2D71200256E7F
:1034000013501A0D840E2524F324156E040EF42097
:10341000146E0CDA376E120002C1DCFF028D2C989C
:103420009B51616E1A0D840EF324136E040EF4206A
:10343000126E01EE62F081D941EC07F066510F0B7C
:103440005D6E63BD63AF21D02C8801EE62F011EE9A
:103450007EF0EEEC06F06639070B7E6FE70E7F1705
:103460006751180B7F1301EE70F011EE88F076ECC7
:1034700018F064EC02F011EE8CF025EC18F011EE6F
:1034800070F025EC18F041EC07F0DDCF02F10EEC06
:1034900006F01200146A540E156E9B51B0D901EE5D
:1034A0002AF002B101EE46F011EE62F0EEEC06F009
:1034B0007D0EF76E2C0EF66E01EE74F095DE649FB5
:1034C000666B676B628FC80E9B6527AF22D001EEDB
:1034D0002AF002A101EE46F011EE7EF0EEEC06F0CD
:1034E0007E39666F7F51180B676F01EE88F015EC1F
:1034F00018F001EE8CF01DEC18F07FBF0EEC02F01E
:103500007FBD19EC02F011EE70F025EC18F0638D20
:10351000638F028D02D8029D12009B511A0D840EFA
:10352000F324156E040EF420146E01EE2AF002B19D
:1035300001EE46F002BD01EE62F021D00CD855D963
:1035400018D810D82A901200500E156E040E146E62
:1035500002EE08F014D0540E156E146A01EE01F05C
:10356000280E0ED05750156E5850146E01EE46F0CE
:1035700006D05350156E5450146E01EE2AF01A0EF8
:10358000256EEE50396E3BD9154A142A252EF9D7EF
:103590001200000E156E1A0E146E01EED0F00C0E15
:1035A000EFD7A00E156E1E0E146E02EE40F0600EE8
:1035B000E7D74F0E156E1E0E146E03EEAFF0510ED0
:1035C000DFD797D8EFEC39F029D99B6F99D889D8F4
:1035D0009FD8A6D82C822C8433D8AB98760EF76E61
:1035E0002E0E11BF04D0020F11BD01D0020FF66ED6
:1035F0000900F5CFB0FF0900F5CFAFFFAB88AE50A3
:10360000AE501200236E2CB8233AF00E2CB80F0ED9
:1036100052142310066F01D812000651521850E0C0
:103620002C922C9406515218256E0F0BD8A42C8284
:103630002550F00BD8A42C842CB29BDF2CB492DF45
:103640002CA21DD006510F0B276E1A0D7D0EF324F0
:10365000136E536E000EF420126E546E6CD81A0E58
:103660005324556E000E5420566E01EE34F0DDDC0E
:1036700028D8446FF7EC07F011EE34F0E6DC2CA408
:103680001DD006390F0B276E1A0D030EF324136E8F
:10369000576E020EF420126E586E4AD81A0E572436
:1036A000596E000E58205A6E01EE50F0BEDC09D85B
:1036B000606FF7EC07F011EE50F0C7DC0651526E68
:1036C00012000E0E2760000C2750F80FD8A0E86AF1
:1036D0001200F80E136E180E126E02EE3CF0040E7D
:1036E0002DD0CF9D500E136E040E126E02EE08F018
:1036F00024D0530E136E126A01EE00F02A0E1ED073
:10370000000E136E1A0E126E01EED0F00C0E16D0D3
:10371000A00E136E1E0E126E02EE40F0600E0ED062
:103720004F0E136E1E0E126E03EEAFF0510E06D04A
:1037300001EE46F002D001EE2AF01A0E256E2506A3
:10374000BDD8A00E83D8125081D813507FD8B5D8D9
:10375000A10E7CD892D8EE6E252EFCD78DD8EF6EB8
:10376000A5D8120009D862E3EF501200396E04D8D0
:10377000395045E3EF6E120014660AD0520E1564FC
:1037800007D07D0E156004D001EE00F0530E1CD062
:10379000040E146206D04F0E156203D001EE9BF0AA
:1037A00015D000EE53F016D806E314D804E201EE6B
:1037B0002AF0535009D000EE57F00CD809E30AD88C
:1037C00007E201EE46F05750155CE926D88012005A
:1037D000D8901200EE50155CEE5014581200CF6BCA
:1037E000790E156E146A26510AD0040E146E4F0E0F
:1037F000156E9B5104D0640E156E146A1151CFA33F
:10380000CFB51200396E12D8395CD8B4120016D870
:1038100039501CD84BD8A8EC01F01200040E146EDD
:103820004F0E156E03D0640E156E146A07D845D876
:10383000A10E0CD821D83AD86D5012003FD8A00E56
:1038400005D8145003D8155001D812006D6E080E1B
:103850006C6E6D36D8B026D8D8A03BD834D86C2E34
:10386000F8D720D83DD838D83BD883AA2C9C83BA27
:103870002C8C2CD835D812002C8E080E6C6E30D8BB
:103880002BD82ED86D3683BA6D8083AA6D901ED842
:103890006C2EF5D72CAE03D005D815D804D019D886
:1038A00012D81ED8958A6D502C9E120012D818D8A6
:1038B00013D816D8F7DF14D81200F8DF0DD8F2DFCE
:1038C0000FD807D802D00CD807D80AD88C9895986A
:1038D00012008C9A959A1200958883A8FED7120040
:1038E000140EFF0FD8A4FDD712006EBC20D06EBE00
:1038F00040D00B50ECD80A50EAD80950E8D808500C
:10390000E6D87250E4D88B82B5D88B921200000EA4
:103910008B92EED800EE72F052D0010E8B92E8D866
:1039200000EE76F04ED0020E35D0030E2ED0040EEF
:103930008B92DED800EE08F042D0050E2BD0060E9A
:10394000F7D7000E8B92D4D800EE72F03ED0010E65
:103950008B92CED800EE73F034D0020E8B92C8D882
:1039600000EE76F030D0030E8B92C2D800EE78F0E5
:1039700028D0040EDDD7050E0DD0060E10D0070E90
:1039800009D0080E11D0090E0FD08B92B1D800EEDD
:1039900013F01BD08B92ACD800EE12F014D08B92A7
:1039A000A7D800EE11F00DD08B92A2D800EE10F047
:1039B00006D08B929DD800EE0FF0EE5099D8EE50C5
:1039C00097D8EE5095D8EE5093D8EE5091D88B8280
:1039D000120082B81BD08B8AA8EC01F082A816D006
:1039E0008B9AA8EC01F082B811D0338A8B926AD8F6
:1039F000829640D882863ED88B823CD88B925DD806
:103A000054EC02F0000E726E74DF2DD05BD8010E04
:103A100081D864EC02F05BEC03F007E12CD0338E2C
:103A20004BD8EBEC18F08DDF1ED0180E116E5BEC4E
:103A300003F001E106D0040E116E5BEC03F01BE114
:103A400000D052EC18F01380010E59D8010E62D844
:103A50005BEC03F010E11390010E51D8338C2CD89D
:103A6000E4EC18F054DF6E503318E00BD8B41200B9
:103A70003382338412003380338233849480A8EC01
:103A800001F012006E44E8447C0B236E33BC06D078
:103A900033BE0BD072906EB272801200030E781695
:103AA000234478126FB0788438D7030E73162350EE
:103AB00073126FB0738E4BD7E1DF949A800EC76E8E
:103AC000300EC66E8B909490A8EC01F01200E83294
:103AD0002336E8322336E8322336E8322336E8321A
:103AE0002336E8322336E8322336E832233400D056
:103AF00033B21200C96EC7A0FED7C95012008B9214
:103B0000000915D8115013D8125011D813500FD8DE
:103B10008B8212008B9280090AD861EC02F017D8D0
:103B2000166E15D8176E13D8186E8B821200949AE1
:103B30006D6E080E6C6E6D36D8B08B8AD8A08B9ADD
:103B40008296CEDE8286CCDE6C2EF5D71200948A69
:103B5000080E6C6E8296C4DE6D3682BA6D8082AAC3
:103B60006D908286BDDE6C2EF5D76D5012007EEC16
:103B700037F02FAED8B00DD0040EB0EC37F093EC88
:103B800037F087EC37F0050E2FB2B0EC37F003ECCE
:103B900014F01E0E256E01EEAAF050EC02F0ACD827
:103BA000020E90EC18F0EFBAAA81EFB8AA8304BB1A
:103BB000AA8504A1AA8704A3AA89EFAAAA8BC8513F
:103BC000AB6F08BDAC8108BFAC8326A1AC8526A332
:103BD000AC8728B3AC8905BFAC8B000E90EC18F015
:103BE000070EEF14AAD8AD6F0F0E5C14AE6F040E63
:103BF00004A1E88004A3E882A0D8AE13000E08BD9B
:103C0000E88008BFE88299D8AF6F040E26A1E8804B
:103C100026A3E88292D8AF13C85101D0B02BE83266
:103C2000D8A0FCD784EC18F0EF38B01384EC18F06F
:103C3000EF5083D8B16F2751B1153F0BD8A4B28193
:103C4000D8B4B28330A2B28530B2B28702BD04D0FC
:103C500002A1B28902B1B28B02BDB28DC79F600EC4
:103C6000266EF29C2F888A848A988A968FEC01F0BF
:103C70008FEC01F08A8612EE9FF0E550CA6FF28C4D
:103C8000070B5BD8C96FCA41E840E8401F0B01EE43
:103C9000A8F0EB50C915D8B48A90D8A48A808FECCC
:103CA00001F0F29C8A948FEC01F00CD88A84262EC5
:103CB000E4D78FEC01F08A948FEC01F08A882F987A
:103CC000F28C120001EE9CF00C0E256E0B0EEB3404
:103CD000EE36252EFDD79C9181BA9C811200A86BEF
:103CE000A96B0F0E5C14010FD880A837A937E82EF6
:103CF000FCD72DBEA98F12000CEC14F0760EF76ED7
:103D0000900EF66E000E90EC18F0EF50070BF626B2
:103D10002F948DEC18F0EFA8EFB602D0200E06D04D
:103D20002F84000E0BBD080F0BBF100FF6260800E6
:103D3000F5502FB2400EC86F1200256A010FD880CF
:103D40002536E82EFDD725501200600E256E02EEB6
:103D500040F0750EF76E000EF66E0900F504EE6E7B
:103D6000010F252EFAD712000101F86A100EC26E5B
:103D7000AA0EC06EC280900EAB6E670EAC6E480E7F
:103D8000B86E51DD116F29DCC30ED56E05EEFFF064
:103D9000ED6AEAA6FDD7C282432AE12B308246684B
:103DA0006B684780616820EE80F0A50EE8CF80F058
:103DB000E8CFBDF0070E286ED08EF194F28AF2940F
:103DC0009F9A9D8A9EBAAE50F28EF28C12008ACFD4
:103DD000DCFF8CCFDCFFFACFDCFF51B2C8D08C8E79
:103DE000CE0E8A128A90B486D9B191D000D000D07C
:103DF00000D000D0B434E237E836E337E099E2513E
:103E0000D8A402D0E09106D0E21DD8A402D0E0816F
:103E100001D0E089E351D8A402D0E09306D0E31D9D
:103E2000D8A402D0E08301D0E089E0A909D0E62B34
:103E3000400EE661E66F320EE66504D0E76902D017
:103E4000E667E607D890E437D890E437E0B1E4813C
:103E5000E0B3E48300EC39F0E56FE7AFE5AD13D0F4
:103E6000DFC1E8F0E151E5B7DF27E5B9DF5F300EEC
:103E7000DF6505D0E86CDF6102D0E8C0DFF1DAC1B0
:103E8000E1F1DB51EA6FE5AB18D0320EE66115D0F7
:103E9000E5A10AD0E82B070EE861E86FE967E907BA
:103EA0002EEC38F040D909D0E92B070EE961E96F13
:103EB000E867E8072EEC38F036D9E087E851E96189
:103EC000E097EA6704D0DB51EA6FE12DE16FEA0782
:103ED000E767E707432E17D1200E436EE7AF16D0F2
:103EE0002EEC38F020D9DFC1E8F0E151E0B7DF2750
:103EF000E0A7DF5F300EDF6505D0E86CDF6102D040
:103F0000E8C0DFF1DAC1E1F1DB51EA6F30D04350B4
:103F1000030BD8A426D003D9D890E233D890E2334B
:103F2000B450C00BE213550EE215D8B4E091550A17
:103F3000D8B4E081AA0EE215D8B4E093AA0AD8B4A6
:103F4000E083E0B50BD0E0A109D0E151E0A3E86C3B
:103F5000DF6F060EE16F2EEC38F0E5D8E095E0B1AA
:103F6000E085432ED0D0200E436EE12DE16FCFB11E
:103F7000CFBD10D0CB2F0ED0CB87CC67CC07CD6771
:103F8000CD07CD6702D0CFB703D0CFA7CC6702D083
:103F90002F80F9D82FA851B29CD0B4968A808A92EB
:103FA000BED8B438B4860C0B496EB9D8B4508A82E6
:103FB0008A94C00B4912B3D8B450B496C00B4A6E61
:103FC000AED8B4388A848A960C0B4A12A8D8B43872
:103FD000B4860C0B4B6EA3D8B4508A868C9EC00B53
:103FE0004B129DD8B450B496C00B4C6E98D8B438D0
:103FF0008C8E8A9C0C0B4C1292D8B438B4860C0B65
:104000004D6E8DD8B4508A8C8A9EC00B4D1287D8C5
:10401000B450B496C00B4E6E82D8B4388A8E0C0B56
:104020004E122D90403C406EE86A4ABE800E49B464
:10403000810E4AB4820E4BB4830E49B6840E4AB642
:10404000850E4BB6860E49BC870E4ABC880E4BBC0B
:10405000890E31A004D049BEAA0E4BBECB0E000F74
:10406000D8A4416ED8B4406A49504A104B104C1045
:104070004D104E1002E057D82D80419E3F3C3F6EC0
:104080004CA43F6A02BD03D0860FD8B42E803E3CBC
:104090003E6E4CAE3E6A3D3C3D6E4CAC3D6A3C3C97
:1040A0003C6E4CA63C6A02BD03D0B40FD8B42E823D
:1040B0003B3C3B6E4BBE03D03B6A2E9E2E9C4B0E70
:1040C0003B5CD8B42E8E960E3B5CD8A402D02E8CCE
:1040D0002E9E423C426E80B8426A472C476E463C58
:1040E000466EFE08D8B42A80010E455E000E445A82
:1040F000D8A02C80483C486E682C686E6B3C6B6E78
:104100008008D8B43080DDCFFAFFDDCF8CFFDDCF63
:104110008AFFF294DDCFD8FFDDCFE8FF1000210E3B
:10412000FF0FFEE11200050E446EF60E456E120002
:10413000E9CFDCFFEACFDCFFAECF69F0684C676AFD
:104140006B6A100E686E00EEC4F06650662466243A
:104150006624662467246AA069C0EBFF672A050EFF
:1041600067620CD0676A6A9066C069F06628030BC4
:10417000666E656203D069C066F06A80DDCFEAFFD3
:10418000DDCFE9FFC7D7D051CFA3D251CC6FD151EA
:08419000CFA3D351CD6F120043
:106D00003182CAEC17F02DA2B6D02DA802D0416670
:106D1000B3D06D0EFA6E41441E0BCFB3140F02BDFB
:106D2000280FCFB5140FF92627D0B1D0DAD024D14F
:106D300024D133D137D137D139D142D192D1A1D158
:106D4000A5D1A5D1A5D1A6D1A6D1A6D1A7D1A9D18A
:106D5000B0D1B0D1B0D1B0D1BED1BED1BED1C5D1EC
:106D6000DED1E7D1FAD1FCD1FCD1FCD100D200D2E6
:106D700000D200D200D202D289EC18F0EFBC7BD056
:106D80002C903180F1EC01F064EC02F0FEEC15F097
:106D90002CA003D001EC02F06ED06FEC16F0CAEC20
:106DA00017F02DA2F5D7030E2FBC040E296E41ACAF
:106DB00013D031B202D02A8E2906FEEC15F02CA099
:106DC00003D001EC02F057D06FEC16F0CAEC17F0CC
:106DD0002DA2F5D741BC2DD041AA08D02ABCEFD7AF
:106DE0002A8C050E2CBA060E296EE7D72950E7E04B
:106DF00029042ABC0DD061EC02F00A0E186E12ECC8
:106E000003F000EE0AF028EC18F0050E2CBA060E7E
:106E100002EC03F041500F0BF9EC02F00EEC02F023
:106E20002ABC05D061EC02F05BEC03F0D8A4290683
:106E3000C4D74BBEFED7BE6BFEEC01F02ABE3AECC7
:106E400002F031A618D02A8016D87FEC18F0EFCFC8
:106E50005BF043EC07F0F1EC01F07FEC18F0EF5041
:106E60005B5ED8B405D002EC1BF0CFA1A4EC17F008
:106E700001EC02F012002D92316A2A9C2A9E120027
:106E80002D92405003E02B08FCE22D821200474C6B
:106E90001BD052502CB852380F0B5C6E5C2A0F0E70
:106EA0005C605C6A66EC37F0D8A0F8D75C5002EC06
:106EB0001BF0A4EC17F014EC18F05C50276EF7EC04
:106EC00007F024EC18F0CAD8476AD5D75C50256E75
:106ED000D75125B6D8512596252AE830252EFDD73D
:106EE0001200472C08D087EC37F0050E2FB2EF6E5A
:106EF00003EC14F0B3D8010E476EBDD7A0EC37F009
:106F00003A28256ED651E830252EFDD71200A0EC88
:106F100037F03A2A070E3A1680EC37F0D8A0F9D7A6
:106F2000A7EC37F01200A0EC37F03A06070E3ABE95
:106F30003A6E80EC37F0D8A0F8D7A7EC37F0120003
:106F4000000E90EC18F0EF50070B3A6E1200000E96
:106F500090EC18F0F80EEF163A50070BEF121200F3
:106F6000E8CFDCFF000E90EC18F0F80EEF16DDCF46
:106F7000E8FF070BEF1212007ED7474CA5D75250FF
:106F80002CB852380F0B5C6E5C060E0E5CBE5C6E4D
:106F900066EC37F0D8A0F8D789D7472CACD793EC5C
:106FA00037F0A3D768D7472C28718DD737D8CF8330
:106FB000E1EC1AF0CF9941EC07F0B6EC17F02CD0C9
:106FC00002EE21F0EFB0EFA256D728D8CF83CF89B9
:106FD00069EC1BF0C80E9B6F0CEC1AF0E7EC06F0A6
:106FE00014EC18F0A4EC17F042EC15F024EC18F0B7
:106FF00002EE3CF015EC18F042EC15F01CEC18F029
:107000005BEC03F005E26BEC18F048EC18F004D0F0
:1070100043EC18F070EC18F035D0CF839EEC1AF0EA
:10702000010E476E0DD806D8080ECB6FC3EC20F0CA
:107030002F901200486A6FEC16F048AEFCD7120091
:107040008C0EB2EC01F01FEC08F0020ED403770EA8
:10705000F76E980EF324D2EC18F01200466A2A90CC
:107060001200EFEC1BF040BE04D04050FCE12A803F
:1070700006D0E1EC1AF071EC1BF041EC07F0DF6B8D
:10708000FAD62695CF8130A2CF91F5D62AD7F3D65E
:107090002685F8D782D7EFD6CF71F5D7CFA9EBD613
:1070A00089D7CFB9E8D602EE21F0EFB0EFA2E3D650
:1070B0008ED7E1D6E0D615D7C70E9B652EA4DBD6BA
:1070C000DFDE2DA204D05CEC0AF042D8D4D6627F79
:1070D0008DEC1AF0D0D6CFD660D7C70E9B652EA404
:1070E000CAD62DEC0AF034D8C6D640BE0AD04050DD
:1070F000FCE1C70E9B652EA4BED6647F8DEC1AF012
:10710000BAD670EC0DF013A007D0C9EC09F0381C0A
:10711000EF162E94A4EC1AF02D981AD8ACD67AEC6F
:1071200009F0CFBD12D07ADFCF85CF997AEC09F084
:10713000A9D77AEC09F0CFBD08D070DFCF897AECFF
:1071400009F0CF8512EC0AF09DD771EC1BF089D7BE
:10715000F29C6650656EF28C120071EC1BF081D7C8
:1071600090D7BFD6CFB9E2EC09F0F2DF8BD790D73A
:1071700014D781D691D7CFA97ED6D7D7CFB97BD612
:02718000DDD759
:10720000720EFA6EE4451E0BF926000C210C220CBE
:10721000040C220C000C040C690C210C040C000C56
:0A722000720C040C220C210C000C6F
:10730000730EFA6E2744F926710C790C810C890CE6
:10731000910C990CA10CA90CB10C1F0C270C2F0C73
:10732000370C3F0C170C730EFA6E2744F926710CBC
:10733000790C810C890C910C990CA10CA90CB10C45
:10734000B90CC10CC90CD10CD90C950C506E730E34
:10735000FA6E50440E0B2CAA020FF926CA0CC90C67
:10736000C80CC60CC50CC40CC20CC10CC00C730EEE
:10737000FA6E000E90EC18F0EF440E0BF926000C9C
:10738000010C020C030C040C02D00A0C0C0C2FA2F2
:10739000080C060C730EFA6E14441E0BF926000C32
:1073A000010C020C030C040C000C050C000C050C69
:1073B000000C060C000C070C000C000C000C519A81
:1073C000519C519E730EFA6E2639060BF92606D093
:1073D00006D002D0518E03D0518C01D0518A268B19
:0473E000269D1200D4
:10740000740EFA6E4F44F926000C96EF16F0010C3C
:10741000A8EF16F0020CC6EF16F0030CC9EF16F039
:10742000050CDFEF16F0070CE2EF16F0080CF5EF95
:1074300016F0090CFBEF16F00A0C08EF17F00B0C16
:1074400009EF17F00C0C0AEF17F00F0C0BEF17F009
:10745000100C12EF17F0800C17EF17F0810C1DEFD6
:1074600017F0820C1FEF17F0850C22EF17F0880C35
:1074700025EF17F08F0C2FEF17F0A70C31EF17F057
:10748000BA0C3CEF17F0BB0C3FEF17F0BC0C48EF09
:1074900017F0BD0C51EF17F0BE0C5BEF17F0E70CC7
:1074A0005CEF17F0F50C61EF17F0F70C72EF17F0C7
:1074B000F90C79EF17F00D0C8BEF17F00E0C8DEF28
:0274C00017F0C3
:1074F00000000240180000F200000000000003023B
:107500000706080504030201090A0F2E2F2B292A5A
:107510002D16531235371325265223240000000060
:10752000000000000000000000000000000000005B
:10753000000000000000000000000000000000004B
:10754000000000000000000000000000000000003B
:10755000000000000000000000000000000000002B
:10760000000927C04E20271013880BB809C407D0E3
:1076100005DC04E203E803840271025801F4012C42
:1076200000FA006403E70098967F05F5E0FF010388
:107630000411082200002710000186A000000000AD
:10764000000000000000EA600007A120000F424097
:10765000FFFFFF6AFFFFFF6A000000960000009630
:10766000000000000000004600000000FFFFFFBA1D
:10767000000000000000000000000000000000000A
:1076800000000000000000000000000000000000FA
:107690000101010104200110020201010420021075
:1076A000010108080420081002020808042008103C
:1076B0000101010104100110E7E7E7E7E7EFE7E761
:1076C000F7F7E7E7E7EFF7E7E7E7F7F7E7EFF7E7DA
:0876D000F7F7F7F7E7EFF7E722
:10770000004C53C2005553C2200043D7004357D208
:10771000202041CD200046CD00414DF300504BD4F8
:10772000205746CD312EB8332EB5372EB02031B08C
:107730002031B42031B82032B12032B42032B82008
:1077400035B02038B83130B83134B43433B02D2DA1
:10775000AD2D2DAD313630ED203830ED203430ED0B
:10776000203330ED203230ED203137ED203135ED52
:10777000203132ED203130ED202036ED202046CD75
:10778000204149D2202032ED373063ED2D2D2DAD33
:107790002D2D2DAD202048C653B053B153B253B355
:1077A00053B453B553B653B753B853B931B032B0DD
:1077B00033B034B035B036B0606060676060606030
:1077C00060606267626060606060717B757171604B
:1077D000606071717F7171606060607E64687E60FE
:1077E000646464647F6E6460646E7F646464646017
:0877F0006060606C6C6060E0F9
:0277F80000008F
:107800005249D45250D4205350CC205458A0202058
:1078100020202058204F4646534554A0204444532E
:10782000A05245462046524551A0204C455645CCD5
:1078300043D75353C2204E4152524F57A02020A04D
:10784000524EC45945D3204ECF2006A02005A03C5F
:1078500006BE3C05BE203DA03C3DBE3C2ABE535466
:1078600045502053495AC52042414E44A04D49CE6F
:107870004D41D8444953504C41D943484950205474
:107880005950C54F2F5020444956494445D2535969
:107890005354454D20434CCB44495649444520421E
:1078A00059A04F5645522D434C4F434B204444530F
:1078B00020BF2A205741524E494E47202A202055AA
:1078C00053C5415420594F5552204F574E205249CD
:1078D00053CB4D554CD44F2F502020202C204655B3
:1078E0004E432E2020A04E4F5420494E5354414C1D
:0778F0004C4544202020A0BC
:107900000203842023A02034B82039B63334B830A1
:107910003020424155C44E4F4E4520202020A041EA
:1079200044393835302F35B14144393935312F3567
:10793000B44144393935382020A04D454D4F525976
:1079400020495320454D505459A053415645205489
:107950004F204D454D20A044454C455445204D45B4
:107960004D4F525920BF2053415645204348414E68
:1079700047455320BF2041524520594F552053556C
:10798000524520BF5646CF4D45CD20535745455013
:107990002054494DC52050415553452054494DC5AB
:1079A000205345C3202048414C5420A05343414E0E
:1079B000204D454D2047524F5550A04E4F54204525
:0B79C0004E4F554748204D454D27D342
:107A000043414C204D454E55A04558495420202017
:107A10002020202020202020A04444532043414CFB
:107A20004942524154494F4EA042414E4420465291
:107A30004551204C494D4954D34444532052414E62
:107A40004745204C494D4954D353204D4554455248
:107A50002043414C20202020A04241434B55502040
:107A600043414C20494E464FA0524553544F524536
:107A7000204241434B555020A05553455220545568
:107A80004E41424C45202020A04C454741435920BF
:107A90002020202020202020A04143432E20202CE5
:107AA0002053454E532E2020A0454E41424C4520A8
:107AB0004154204C45415354A04F4E452053454C12
:107AC000454354494F4E2020A0534156494EC7507C
:107AD00048414E544FCD4F55542D424EC4535441FE
:0B7AE00054494F4E204C4556454CA029
:107B00005345545550204D454E55A0455849542095
:107B100020202020202020202020A04D4F44204D38
:107B20004F4445204F4646534554D3484944452089
:107B30004D4F44204D4F44455320A04849444520D3
:107B400042414E44532020202020A0492F4F204264
:107B50004F415244205345545550A0524F54415226
:107B60005920454E434F44455220A0535745455058
:107B700020534554555020202020A04241554420F8
:107B800052415445202020202020A04F5054494FDE
:107B90004E414C2046494C544552D34C4F41442011
:107BA00044454641554C54532020A0454E41424C3B
:107BB000452053454C454354494FCE484944452000
:107BC00053454C454354494F4E20A04F462020205A
:107BD00020204D4F44204D4F4445A04F462054484F
:0B7BE0004520202020202042414EC400
:107C000046554E4354494F4E204D454E55A045587C
:107C100049542020202020202020202020A0505225
:107C200045414D50202020202020202020A04E4FD4
:107C300049534520424C414E4B45522020A04154CF
:107C400054454E5541544F522020202020A04147FA
:107C500043202020202020202020202020A04E4132
:107C600052524F572046494C5445522020A04F5560
:107C70005450555420504F574552202020A0535067
:107C8000454543482050524F434553534FD2564FDA
:107C900058202020202020202020202020A0414EDD
:107CA00054454E4E412020202020202020A04C432F
:107CB00044204241434B4C494748542020A04F4662
:107CC00046A04C4F57A04D4544A0484947C84F4E89
:107CD00020A04F4646A0534C4FD7464153D4415560
:027CE00054CF7F
:107D0000414E54203120285265617229202020A044
:107D1000414E542032202846726F6E74292020A0D4
:107D2000207820524546434C4B2020A04D454D2DF8
:107D30002D5441474D696E692D4B697473A04D31C7
:0C7D400020524144494F2076312E4BA0C8
:020000040030CA
:0100010046B8
:010002000EEF
:0100030000FC
:010005008179
:010006008178
:010008000FE8
:010009008076
:01000A000FE6
:01000B00A054
:01000C000FE4
:01000D0000F2
:0200000400F00A
:1000000026000000002DC6C000EE9BFAB4006ACFA7
:10001000C00000000000000000271000325AA000BD
:10002000325AA10073F7800073F78100A4CB8000DF
:10003000A4CB8100DA336000DA3361010B07600280
:1000400080DE8002CD29C0000DBBA00000000000B2
:100050000000000000000000000000FD8E63C00DE5
:10006000BBA0000000000000000000000000000035
:10007000000002BF2000030D400005573000061AA3
:1000800080000AAE60000B2390000F6950000F7CC7
:10009000D800155CC00015E578001B91D0001BB896
:1000A000E0002032300020BAE80025FAA80026211E
:1000B000B8002AB980002D5190004C4B4000526589
:1000C000C00086470000A4CB8000A4CB8100D10BE8
:1000D000A000DBBA0000E1D4800280DE8002AEA581
:1000E00040003F007F00BF00FF013F017F01BF01D3
:1000F000FF023F027F02BF02FF033F037F03BF00F7
:00000001FF
